:100000000C9463110C94B2110C94B2110C94B211B3
:100010000C94B2110C94B2110C94B2110C94B21154
:100020000C94B2110C94B2110C94172C0C94B211C4
:100030000C9488220C94B2110C94B2110C94B2114D
:100040000C94B2110C94F5260C94B2110C94B211CC
:100050000C94B2110C94B2110C94B2110C94B21114
:100060000C94B2110C94B2110C94B2110C94B21104
:100070000C94B2110C94B2110C94B2110C94B211F4
:100080000C94B2110C94B2110C94B2110C94B211E4
:100090000C94B2110C94B2110C94B2110C94B211D4
:1000A0000C94B2110C94B2110C94B2117619BF14C5
:1000B000C514E714ED14151670169E1619179B1724
:1000C000D317A918FB181F191615381554156E15D6
:1000D0008315D915CF16E116EA16F516FE16D816B1
:1000E0003819501964190D18231836184C185D1852
:1000F0006F1883189718251628162E1638163E16D0
:1001000041164716521658165B162E1661166716BC
:100110002D173017361739173F1747174D17581730
:100120005E17611767176A17701778177E1785179C
:100130008B17E317E817ED17F217F717FC170118DD
:100140000618BC18BF18C618C918CF18DA18E01856
:10015000FF2C262D0F2E262D0F2E712D922D0F2EBA
:10016000E52DF42D0000000000000000000000005C
:10017000000000002A002B002800000000002800DA
:10018000000000000000000000000000000000006F
:100190000000000000000000000029000000000036
:1001A000000000002C001E02340220022102220264
:1001B000240234002602270225022E0236002D00DA
:1001C0003700380027001E001F00200021002200F9
:1001D00023002400250026003302330036022E00BF
:1001E000370238021F020402050206020702080253
:1001F00009020A020B020C020D020E020F0210028B
:10020000110212021302140215021602170218023A
:1002100019021A021B021C021D022F0031003000BD
:1002200023022D0235000400050006000700080027
:1002300009000A000B000C000D000E000F0010005A
:10024000110012001300140015001600170018000A
:1002500019001A001B001C001D002F023102300281
:1002600035024C000000000000000000000000000B
:10027000000000000000000000000000000000007E
:10028000000000000000000000000000000000006E
:10029000000000000000000000000000000000005E
:1002A000000000000000000000000000000000004E
:100590000000000002000000000000000000020057
:1005A000000000000000000000000000000000004B
:1005B000000000000000000000000000000000003B
:1005C000000000000000000000000000000000002B
:1005D000000000000000000000000000000000001B
:100840000000000000351E1F20212223242526271A
:100850002D2E2A002B141A0815171C180C12132FF2
:1008600030000029041607090A0B0D0E0F3334322D
:100870002800E1641D1B061905111036373800E504
:1008800000E0F1E200002C00000000E6F265E40068
:100890000000000000000000000000000000000058
:1008A0000000000000000000000000000000000048
:1008B000000000005051524F0000000000000000F6
:1008C0000000000000000000000000000000000028
:1008D0000000000000000000000000000000000018
:1008E0000000000000000000000000000000000008
:1008F00000000000000000000000000000000000F8
:100B3000000000FF07FF07FF07FF07FF07FF07FF92
:100B400007FF07FF07FF07FF07FF07FF07FF07FF75
:100B500007FF070000000000000000000000000088
:100B60000000000000000000000000000000000085
:100B70000000000000000000000000000000000075
:100B80000000000000000000000000000000000065
:100B90000000000000000000000000000000000055
:101B300000000001010000000000000000000000A3
:101B40000000000000000000000000000000000095
:101B50000000000000000000000000000000000085
:101B60000000000000000000000000000000000075
:101B70000000000000000000000000000000000065
:101B80000000000000000000000000000000000055
:101B90000000000000000000000000000000000045
:101BA0000000000000000000000000000000000035
:101BB0000000000000000000000000000000000025
:101BC0000000000000000000000000000000000015
:101BD0000000000000000000000000000000000005
:101BE00000000000000000000000000000000000F5
:101BF00000000000000000000000000000000000E5
:101C000000000000000000000000000000000000D4
:101C100000000000000000000000000000000000C4
:101C200000000000000000000000000000000000B4
:101C300000000000010000000000000000000000A3
:101C400000000002FF000000FF00FF00FF00FF0097
:101C5000FF00FF00FF00FF00FF00FF00FF00FF008C
:101C6000FF00FF00FF00FF00FF00FF00FF00FF007C
:101C7000000201000600000000000000000000005B
:101C80000000000000000000000000000000000054
:101C90000000000000000000000000000000000044
:101CA000010204010402034001800140008002108F
:101CB0000002000100200010028002400008000025
:101CC00000002E000000002D000000002B0000008E
:101CD0000027000000000F000000000000000000CE
:101CE00000000000000000000000000000000000F4
:101CF00000000000000000000000000000000000E4
:101D00000000000000000000000000BB00C000FF59
:101D10002F400003000E05010081222A25562500D0
:101D200000000081222F257A13A714000042797445
:101D300065732028686578293E20004164647265D7
:101D400073732028686578293E200020532D307851
:101D5000005D20432D3078000A5B004F7574206FC2
:101D6000662072616E67652E0A00496E76616C6945
:101D7000642073656C656374696F6E2E0A003A2087
:101D80004F4646003A204F4E00205B312D31365DE4
:101D90003E2000205B312D3235355D3E2000205B3A
:101DA000312D3939395D3E2000205B312D39395DC7
:101DB0003E2000205B302D395D3E2000205B303D11
:101DC0004F46462C20313D4F4E5D3E2000205B317A
:101DD0002D345D3E200044656661756C742042615F
:101DE000636B6C69676874204D6F64650044656659
:101DF00061756C74204261636B6C6967687420451F
:101E00006E61626C650044656661756C742044693E
:101E10006D6D6572204C6576656C004D61747269FC
:101E20007820536574757020576169742028637930
:101E3000636C65732900526570656174205065722A
:101E4000696F6420286D7329004D696E20486F6C9E
:101E5000642054696D6520666F72205265706561FB
:101E60007420286D7329004D6F757365204D6F7652
:101E7000656D656E74204D756C7469706C69657202
:101E80000042617365204D6F757365204D6F7665F7
:101E90006D656E74004D61782044656C61792054E5
:101EA000696D6520666F7220446F75626C652054A1
:101EB000617020286D7329004D617820486F6C6433
:101EC0002054696D6520666F722054617020286D02
:101ED0007329004465626F756E63652054696D6592
:101EE00020286D732900416C7465726E61746520E1
:101EF0004465626F756E6365205374796C65005537
:101F00006E6C696E6B6564204E756D204C6F636BF3
:101F100000426F6F74204B6579626F617264004498
:101F2000656661756C74204C617965720057696EE5
:101F3000204C6F636B206F6E205363726F6C6C204C
:101F40004C6F636B005669727475616C204E756DD1
:101F500020506164000A3929204261636B0A3E20E7
:101F6000000A382920000A372920000A36292000D3
:101F70000A352920000A342920000A332920000AC2
:101F8000322920000A312920000A4C4544204D65A1
:101F90006E753A000A54696D696E67204D656E75FD
:101FA0003A000A436F6E666967204D656E753A00A8
:101FB0000A4465627567204D656E753A0A312920BD
:101FC0005072696E74206576656E74730A322920CA
:101FD000436C656172206576656E74730A332920DF
:101FE0004578616D696E65206D656D6F72790A3433
:101FF00029205072696E742F636C65617220636C66
:102000006F636B2D696E730A3929204261636B0A15
:102010003E20000A4D61696E204D656E753A0A31A9
:102020002920436F6E666967206D656E750A3229D7
:102030002054696D696E67206D656E750A332920BD
:102040004C4544206D656E750A34292044656275DF
:1020500067206D656E750A35292052657365740AAF
:10206000392920517569740A3E20001E4D1F5120E8
:102070004E21502200234F244A2552264B27493710
:102080004CB500B600B700CD006F007000E200E56F
:1020900000E900EA00520153015401550183018A0D
:1020A0000192019401210223022402250226022723
:1020B000022A02B101B202B304B408B510E001E192
:1020C00002E204E308E410E520E640E780010508A9
:1020D0000A0C0F10141418180038330400013D04C2
:1020E00001014104020131040301380404014004E8
:1020F00005014204060134040701370408013A04CB
:10210000090235040B0232040D0139040E013E04AC
:102110000F02300411013C0412012E0413012F049C
:1021200014014A0345006100730079004100560024
:10213000520020004D0075006C00740069006D00B5
:10214000650064006900610020004B0065007900B3
:1021500062006F00610072006400200076003300AE
:102160002E00300031002E0031003000000004034A
:10217000090409026D00040100A0FA09040000012D
:10218000030101000921B00100012240000705817F
:10219000030800010904010001030000000921B047
:1021A000010001223200070582030300080904022E
:1021B0000001030000000921B001000122270007EF
:1021C0000583030E00010904030001030102000955
:1021D00021B0010001223A00070584030300051223
:1021E00001000200000008EB03FF201000000100C6
:1021F00001050C0901A1018502160100269C021AA5
:1022000001002A9C02751095018100C0050109801A
:10221000A10185031981298375019503810695051F
:102220008101C005010902A1010901A100050919E7
:10223000012903150025019503750181029501759A
:102240000581010501093009311681FF267F00361D
:102250000000460000950275088106C0C00501090E
:1022600006A101050719E029E7150025017501956B
:102270000881021500250105071900296795687571
:10228000018102C005010906A101050719E029E73E
:1022900015002501750195088102950175088101D8
:1022A0000508190129059505750191029501750328
:1022B0009101150026FF000507190029FF950675F5
:1022C000088100C00F00EBEEF4E085EC9AE001C05D
:1022D0008193EF3FF907E0F3D9F311241FBECFEF4D
:1022E000DAE0DEBFCDBFC4B714BE0FB6F894A89530
:1022F00080916000886180936000109260000FBE42
:10230000C3FF11C08091E9049091EA048D3A9E4D7B
:1023100051F41092EA041092E904E8EDF0E22591FC
:102320003491F901099585B7806885BF85B78068C4
:1023300085BFC093E80411E0A0E0B1E0E0E3F2E67D
:1023400002C005900D92AE35B107D9F724E0AEE595
:10235000B1E001C01D92A436B207E1F70E949530AA
:102360000C9416310C94000010926C0110926B01C9
:10237000109267011092660110927501109274011B
:10238000089590916A0380916503892B909164036D
:10239000892B90916303892B20916801222309F4F2
:1023A0005FC0811164C080916A01811155C0809124
:1023B000860181113CC090916101921305C0109279
:1023C0006801109261010895E92FF0E0EE0FFF1F00
:1023D000EA58FE4F80812181813031F420936A01D7
:1023E0009F5F90936101089590916201921731F07F
:1023F0002093620181E080936A03089580938601AF
:10240000181614F4E5D70DC099E6980F993118F411
:102410000E94D31A06C093E4980F933010F40E94E0
:10242000021B809161018F5F80936101089587FD98
:1024300003C00E94201A0DC099E6980F993118F434
:102440000E94EA1A06C093E4980F933010F40E9499
:102450000F1B109286010895815080936A010895A0
:10246000811105C0809169018D7F80936901089574
:1024700080916D0290916301981731F1809363010F
:10248000882311F1883211F0883531F48091690187
:102490008B7F809369010895E09165018A3251F440
:1024A000EE2391F0E150E0936501F0E0E359FE4F37
:1024B00010820895E63040F4AE2FB0E0A359BE4F2D
:1024C0008C93EF5FE093650108951092620181E0C3
:1024D00080936A0380916D02811102C0109269019C
:1024E0000895BC0180916801DB01982F292F281BDA
:1024F000983058F090936801620F711D27FD7A950E
:10250000709375016093740122C0FD01259134918F
:10251000211109C090936801109275011092740105
:102520009923D1F014C0492F50E0F901FF27EE0F95
:10253000FF1FEC59FE4F25913491440F551FFA01AE
:10254000EA58FE4F318320839F5F1196CFCF809151
:10255000690183608093690181E008954091680179
:1025600028E030E0241B31092617370758F1B0E086
:102570004B2F0B2E000C550B46175707D8F4A09184
:1025800068012A2F30E0FC01E40FF51FE081F0E044
:10259000EE0FFF1FEC59FE4F45915491220F331F50
:1025A000F901EA58FE4F51834083AF5FA093680161
:1025B000BF5FDECF672B41F080916901836080931C
:1025C000690102C080E0089581E00895909168015A
:1025D000983090F4E92FF0E0EE0FFF1FEA58FE4F1D
:1025E000808361839F5F909368018091690183601C
:1025F0008093690181E0089580E008959C019091A5
:10260000680191112EC0A901983049F49093680196
:10261000205F3F4F30936C0120936B011BC0FA0188
:10262000659174914E5F5F4F6115710549F4909308
:10263000680110926C0110926B01992381F00AC01D
:10264000E92FF0E0EE0FFF1FEA58FE4F7183608321
:102650009F5FDACF8091690183608093690181E097
:10266000089580E00895AC018091680181113EC019
:1026700060937301282F082E000C330B26173707A1
:1026800058F590916801220F331F983038F0240FCD
:10269000351F30936701209366011EC0FA01E20FD7
:1026A000F31F20813181E92FF0E0EE0FFF1FEA5880
:1026B000FE4F318320839F5F909368019091730157
:1026C000915090937301911105C01092670110927F
:1026D000660102C08F5FCECF80916801882341F0F0
:1026E0008091690183608093690102C080E0089550
:1026F00081E0089590916901992329F191FD41CEDE
:1027000020916B0130916C012115310511F0C90147
:1027100075CF20916601309167012115310539F09F
:1027200060917301062E000C770BC9019CCF20919C
:102730007401309175012115310511F0C901D1CE17
:1027400092FD96CEC2CE0895EDE6F1E010821182A0
:1027500012821382148215821092650180916D029B
:102760008093630180916901856080936901089578
:1027700008959091BD01903178F4E92FF0E09F0128
:10278000220F331FE20FF31FE757FE4F8083728340
:1027900061839F5F9093BD01089541111BC04091DB
:1027A000BD0150E090E0292F092E000C330B2417B7
:1027B000350784F4F901EE0FFF1F2E0F3F1FF901BB
:1027C000E757FE4F2081281303C072836183089569
:1027D0009F5FE9CFCECF8A3010F4805D0895895C89
:1027E00008951F93CF93DF93182FEB0182958F707D
:1027F000F2DF8883812F8F70EEDF8983DF91CF91A5
:102800001F9108951F93CF93DF93182FEB01892F0A
:10281000E8DFBE016E5F7F4F812FDF91CF911F9167
:10282000E0CF8F929F92AF92BF92CF92DF92EF92C2
:10283000FF920F931F93CF93DF931F92CDB7DEB715
:102840009C018B0180E3FB01808380E28183828392
:1028500083E0E82EF12C94E6892E912C4AE0B42EE8
:10286000682D70E0911003C02617370790F06801BB
:10287000C90CD11C97FCDA94C9010E94A830A82E7B
:10288000862F9983A8DFF60180832A2D9981392F1D
:102890009394882D6B2D0E949C30882EF1E0EF1AC6
:1028A000F108F1F60F90DF91CF911F910F91FF90FA
:1028B000EF90DF90CF90BF90AF909F908F90089552
:1028C00097EA980F993010F48855089592EE980F72
:1028D000993010F48D5108959CEF980F963010F4B4
:1028E0008A5F089580E00895BF92CF92DF92EF92C1
:1028F000FF920F931F93CF93DF937C018B0180E0B6
:1029000090E0B12CC42FD0E02B2D0B2C000C330BFE
:102910002017310790F48C9F60018D9FD00C9C9FF5
:10292000D00C1124F701E20FF31F8081C9DF96015B
:10293000280F311DC901B394E7CFDF91CF911F91CB
:102940000F91FF90EF90DF90CF90BF9008950F937D
:102950001F93CF93DF9300D000D0CDB7DEB7809127
:1029600069018111C3C4E09187018E2F90E0853207
:102970009105A8F4FC01EA5AFF4F0C94BC3083E1A6
:1029800090E2AFDDE1DE82E088C411E010938701C0
:102990001092880180916D0193DF893019F41092B3
:1029A0008701A4C4853019F41093BE019FC48130FF
:1029B00011F485E072C4823009F443C3833009F412
:1029C0006BC4843009F43FC08AE69DE12DC480EBDE
:1029D0009FE187DDB9DE84E060C483E080938701F6
:1029E00080916D016DDF893011F481E056C4813032
:1029F00011F48EE052C4823069F4E9E8F1E010820B
:102A000012821182339641E0E93BF407C1F710923C
:102A1000BD016CC4833031F48BE39DE162DD94DE53
:102A200081E13BC4843081F683E137C48091880121
:102A300080315CF0109288018AE0898361E070E067
:102A4000CE0101968BDD83E028C488E59DE149DD58
:102A5000BE016F5F7F4F80918801C3DE62E070E04E
:102A6000CE0101967BDD81E59DE13BDD8FE015C464
:102A700080918801082E000C990BFC01EE0FFF1FBE
:102A80008E0F9F1FFC01E757FE4FBE016F5F7F4F08
:102A90008081A7DE62E070E0CE0101965FDD8BE40D
:102AA0009DE11FDD80E1F9C380918801082E000CB3
:102AB000990BFC01EE0FFF1F8E0F9F1FFC01E757C4
:102AC000FE4FBE016F5F7F4F818192819BDE64E08C
:102AD00070E0CE01019642DD8EE085C36091650114
:102AE00070E040E18DE691E0FFDE9093BA018093C3
:102AF000B9011092BC011092BB018DE29DE1F1DCA5
:102B000023DE82E1CAC38091BB019091BC01892B75
:102B100089F40091B9011091BA016091650170E0EA
:102B200040E18DE691E0E0DE800F911F9093BC01C3
:102B30008093BB0110E20AE0E091B901F091BA0183
:102B40008091BB019091BC01E817F907D8F4BE0150
:102B50006F5F7F4F808145DE8091BB019091BC010A
:102B600001972091B9013091BA012817390711F462
:102B70000B8301C01B8363E070E0CE010196EEDCA5
:102B800081110DC02091B9013091BA018091BB0132
:102B90009091BC012817390708F055CFA7C3809141
:102BA000B9019091BA0101969093BA018093B9014D
:102BB000C3CF809188018A307CF0109288018AE02E
:102BC000898361E070E0CE010196C8DC83E08093E8
:102BD00087010E9418278AC3182F117817FF03C096
:102BE00011501E6F1F5F87FD8F5F082F0595111114
:102BF00002C08AE001C080E2898361E070E0CE011A
:102C00000196ACDC85E01802F0011124E00FF11D03
:102C100007FDFA95EE0FFF1FEC5BFB4FBE016F5FE8
:102C20007F4F80819181EEDDC2C2E09188018E2FBD
:102C3000EE0F990BAA0BBB0B8D30910508F04AC023
:102C4000FC01E558FF4F0C94BC3082EA9FE19CC226
:102C500084E89FE146DC85E49FE196C280913404DC
:102C6000882319F084E89DE18FC28EE79DE18CC234
:102C70008FE79FE136DC8DE29FE186C280913D04C3
:102C8000EFCF8AE79FE12DDC8FE19FE17DC28AE3F0
:102C9000898380E28A8380913104BE016D5F7F4F1A
:102CA00090E095C285E79FE11CDC81E19FE16CC269
:102CB00080914004D5CF80E79FE113DC8FEF9EE148
:102CC00063C28BE69FE10DDC86EE9EE15DC28091E2
:102CD0002E04C6CF85E59FE104DC36DD86E083C2A5
:102CE00087E08093870180916D01EADD8093880100
:102CF000893009F47ACE813019F485E49FE194C2D9
:102D0000823019F48DE29FE18FC2833019F48FE194
:102D10009FE18AC2843019F481E19FE185C2853048
:102D200019F48FEF9EE180C2863019F486EE9EE1A1
:102D30007BC28AE69DE1D5DB85E07CC2809188017B
:102D40008330C9F04CF4813089F0823019F58CEB76
:102D50009DE1C7DB85E11FC08530B9F08CF086307E
:102D6000C9F48CEB9DE1BDDB89E115C08CEB9DE1E5
:102D7000B8DB84E110C083EB9DE1B3DB86E10BC0DF
:102D80008CEB9DE1AEDB87E106C08CEB9DE1A9DB1E
:102D900088E101C085E080938701D6DC4DC2809137
:102DA0006D018EDD823048F48093410482E01AC0C8
:102DB00080916D0185DD823050F18BE59DE191DBE5
:102DC000F8CD80916D017CDD8230B8F780933D04B1
:102DD00081E008C080916D0173DD8A3070F78093C7
:102DE000310483E00E943B26E4CD80916D0168DDD3
:102DF000823018F78093400485E0F4CF80916D0114
:102E00005FDD8230D0F68093340487E0EBCF80938F
:102E10002E0480E10E943B2680912E04882321F01D
:102E200086E080934204DECF8CE08093420486E00B
:102E3000D9CF8AE3898380E28A83E09188018E2F4B
:102E4000EE0F990BAA0BBB0B8131910508F06DC0F9
:102E5000FC01E857FF4F0C94BC3084E99FE194C11A
:102E600084E89FE13EDB83ED9EE18EC180914204C8
:102E700047C08FE79FE135DB88EB9EE185C1BE014E
:102E80006D5F7F4F80913A0490913B044AC08AE77E
:102E90009FE127DB85E99EE177C180913504909120
:102EA0003604BE016D5F7F4F91958195910939C0C0
:102EB00085E79FE116DB81E89EE166C180913204DF
:102EC0001FC080E79FE10DDB87E69EE15DC1809139
:102ED000390416C08BE69FE104DB89E49EE154C10E
:102EE000BE016D5F7F4F80913E0490913F0419C0F9
:102EF00086E69FE1F6DA86E39EE146C180913004E2
:102F0000BE016D5F7F4F90E051C181E69FE1E9DA3C
:102F10008BE19EE139C180913C04BE016D5F7F4F22
:102F200090E07FDC65E070E055C185E59FE1D9DA8E
:102F30000BDC89E058C18AE08093870180916D01A4
:102F4000BFDC80938801893009F44FCD813019F4BA
:102F500083ED9EE169C1823019F488EB9EE164C182
:102F6000833019F485E99EE15FC1843019F481E86A
:102F70009EE15AC1853019F487E69EE155C186303D
:102F800019F489E49EE150C1873019F486E39EE18B
:102F90004BC1883019F48BE19EE146C18AE69DE180
:102FA000A0DA88E047C1E09188018E2FEE0F990BDF
:102FB000AA0BBB0BFC013197E830F10560F5E75631
:102FC000FF4F0C94BC3089EA9DE18BDA8DE1E3CEB2
:102FD0008EE99DE186DA8EE1DECE8EE99DE181DA31
:102FE0008FE1D9CE89EA9DE17CDA80E2D4CE89EA0C
:102FF0009DE177DA81E2CFCE8EE99DE172DA82E25D
:10300000CACE89EA9DE16DDA83E2C5CE83E99DE10E
:1030100068DA84E2C0CE88E0BECE6091650170E0DF
:103020004AE08DE691E060DC9C01215031092336B5
:10303000310520F48093420486E076C08BE59DE163
:1030400050DA88E02AC16091650170E04AE08DE6BF
:1030500091E04ADC9C0121503109273E334070F752
:1030600090933B0480933A0489E05EC060916501CF
:1030700070E04AE08DE691E037DC9C012150310997
:10308000273E3340D8F69195819591099093360467
:10309000809335048AE048C06091650170E04AE0A1
:1030A0008DE691E021DC9C01215031092336310568
:1030B00028F6809332048BE037C06091650170E0A0
:1030C0004AE08DE691E010DC9C0121503109233665
:1030D000310508F0B3CF809339048CE025C06091AE
:1030E000650170E04AE08DE691E0FEDB9C01215035
:1030F0003109273E334008F0A1CF90933F048093DD
:103100003E048DE011C06091650170E04AE08DE6FB
:1031100091E0EADB9C01215031092336310508F0AA
:103120008DCF809330048EE00E943B268ACF609141
:10313000650170E04AE08DE691E0D6DB9C0121500C
:1031400031092F3F310508F079CF80933C048FE09F
:10315000EBCF8AE3898380E28A83E09188018E2F16
:10316000EE0F990BAA0BBB0B87309105B8F5FC014C
:10317000EF55FF4F0C94BC3089E89FE105C084E80F
:103180009FE1AFD986E09EE1ACD92FC08091380491
:10319000B7CE8FE79FE1A5D98DEE9DE1F5CF809168
:1031A000370490E0BE016D5F7F4F01963ADB64E02B
:1031B00070E010C08AE79FE194D986ED9DE1E4CFED
:1031C00080912F0490E0BE016D5F7F4F019629DB57
:1031D00063E070E0CE010196C1D907C085E59FE1AB
:1031E00080D9B2DA8CE080938701809188018F5F6B
:1031F000809388017BC08DE08093870180916D0171
:103200005FDB80938801893009F4EFCB813019F4BA
:1032100086E09EE109C0823019F48DEE9DE104C084
:10322000833021F486ED9DE15CD960C08AE69DE1A2
:1032300058D98BE0809387011092880157C0809104
:103240008801823049F0833061F0813079F489E877
:103250009DE147D98AE19FCD89E89DE142D98BE183
:103260009ACD8DEC9DE13DD98CE195CD8BE093CD50
:103270006091650170E04AE08DE691E035DB9C01EC
:10328000215031092031310520F48093380484E045
:1032900018C08BE59DE125D98BE08093870126C07E
:1032A0006091650170E04AE08DE691E01DDB9C01D4
:1032B000215031092031310560F781508093370466
:1032C00088E00E943B26E8CF6091650170E04AE00B
:1032D0008DE691E009DB9C01215031092430310554
:1032E000C0F6815080932F0481E1EBCF0F900F90B7
:1032F0000F900F90DF91CF911F910F91089526E0CD
:10330000829FC0011124FC01E05CFE4F0190F0811E
:10331000E02D208181E090E001C0880F6A95EAF7F6
:10332000822B8083089526E0829FC0011124FC0136
:10333000E05CFE4F0190F081E02D80816095682374
:10334000462B4083089526E0829FC0011124FC0192
:10335000E05CFE4F0280F381E02D208181E090E06F
:1033600001C0880F6A95EAF7822B8083089526E0D2
:10337000829FC0011124FC01E05CFE4F0280F381BA
:10338000E02D208181E090E001C0880F6A95EAF786
:10339000809582238083089526E0829FC0011124B6
:1033A000FC01E05CFE4F0280F381E02D8081682308
:1033B000462B4083089526E0829FC0011124FC0122
:1033C000E05CFE4F0480F581E02D80818623089526
:1033D000E82FE695E695E695F0E0E05AFD4F982F48
:1033E000977021E030E001C0220F9A95EAF79081B2
:1033F000292B208391E09093650390915A0220E05D
:1034000029175CF4E22F022E000CFF0BE359FD4F4D
:1034100030813817A1F02F5FF3CF96305CF4E92F9D
:10342000092E000CFF0BE359FD4F80839F5F9093A3
:103430005A0208951092730281E0809369030895FF
:10344000E82FE695E695E695F0E0E05AFD4F982FD7
:10345000977021E030E001C0220F9A95EAF720959D
:1034600090812923208391E09093650390915A02E3
:103470004DE652E0FA012E2F241B291724F4319136
:103480003813F9CF01C00895E22F022E000CFF0B74
:10349000E359FD4F818180832F5F2917ACF3915051
:1034A00090935A02109269030895E82FE695E695E5
:1034B000E695F0E0E05AFD4F982F977021E030E05C
:1034C00001C0220F9A95EAF790812927208391E085
:1034D0009093650390915A024DE652E0FA012E2F27
:1034E000241B291724F431913813F9CF13C09630D7
:1034F0005CF4E92F092E000CFF0BE359FD4F80838C
:103500009F5F90935A0208951092730281E0809316
:1035100069030895E22F022E000CFF0BE359FD4FC3
:10352000818180832F5F2917ACF3915090935A02C9
:103530001092690308959091150394305CF4E92F7B
:10354000092E000CFF0BE55AFD4F80839F5F90937F
:103550001503089540E060E070E082E41ED9109207
:103560005F020895209115034BE552E0FA019E2F6A
:10357000941B92179CF431913813F9CF921751F0A4
:10358000E92F092E000CFF0BE55AFD4F8181808346
:103590009F5FF4CF9150909315030895682F70E0CA
:1035A00040E083E4FAC82091160330911703232BDF
:1035B00069F48759E82FF0E0EE0FFF1FEF57FF4D3A
:1035C00085919491909317038093160381E08093E3
:1035D000640308958759E82FF0E0EE0FFF1FEF57BF
:1035E000FF4D859194912091160330911703281770
:1035F000390721F4109217031092160381E080938B
:103600006403089593E4980F81E001C0880F9A95B0
:10361000EAF780936E0381E080936303089510922C
:103620006E0381E080936303089580913104809359
:103630006D0308959FE0899F600D112480915502CC
:1036400068130DC080913504909136048417950756
:1036500034F480916C038F5F80936C030895109213
:10366000550210926C030895E0913A04F0913B04E6
:103670004E175F0754F491E0F9019083FFE08F9FAC
:10368000600D1124609355020895F9011082109283
:10369000550210926C03089590917301E92FEE0F7B
:1036A000FF0BEB58FD4F2091570230E0322F2227BD
:1036B000282B3183208381E0890F8093730180352B
:1036C00034F0109268038093640180E185C5089509
:1036D00090916F03911111C0805D803170F4E82FDB
:1036E000F0E0EE0FFF1FED5CF44F85919491880F91
:1036F000991F8D5C944F0C94FE120895CF93DF9325
:10370000C82FD62F80916D03882311F08B5F64D56D
:1037100080E18C0F80936D030EDF80916D03882311
:1037200011F08B5F39D590916D038091310498171A
:1037300011F08FE031D580916D0390915602D0FF4A
:1037400002C0981308C0981308C080916C038111BF
:1037500004C08091310480935602DF91CF91089587
:10376000E82FF0E0EC59FD4F8491882311F060E0E0
:10377000C5CF08950F931F93CF93DF9300D01F926F
:10378000CDB7DEB7082F10E1180F80916D038823A5
:1037900041F08B5F2B834A8369831ED569814A81FF
:1037A0002B81222389F180916D0381132DC080919B
:1037B0006C03882319F061FD109356028091590221
:1037C000801322C062FF20C08FEF840F873620F461
:1037D00060915702842F16C0842F807E803EA1F412
:1037E000E42FF0E0EE0FFF1FE250F14E8491809540
:1037F0009091570289238093570281E080936A0356
:10380000649180E00E94E612812FACDEE091150306
:10381000E11103C08091560206C00E2E000CFF0B72
:10382000E65AFD4F808180936D0380916D0388235C
:1038300011F08B5FB1D490916D0380913104981396
:1038400009C08FE00F900F900F90DF91CF911F91E3
:103850000F91C2C40F900F900F90DF91CF911F91E5
:103860000F910895E82FF0E0EC59FD4F84918823E3
:1038700021F020E040E060E07DCF08956F7062307D
:1038800051F028F4662339F06130E1F00895643096
:1038900011F0683011F5E82FF0E0EE0FFF1FE25055
:1038A000F14EE49180915702E82BE093570280910A
:1038B0006B03882319F0E777E093570281E0809348
:1038C0006A030895E82FF0E0EE0FFF1FE250F14E7B
:1038D000E49180915702E827E8CF08956F70623035
:1038E00009F447C020F4662309F437C00895643012
:1038F00019F0683091F10895E82FF0E0EE0FFF1F06
:10390000E250F14EE491E095609157026E2360938E
:10391000570291E090936A03222309F44BC09091DF
:103920005902981347C08FEF840F873610F4842F05
:1039300012C0842F807E803E09F03CC0E42FF0E06E
:10394000EE0FFF1FE250F14E849180956823609343
:103950005702649180E00C94E612E82FF0E0EE0F3D
:10396000FF1FE250F14EE491E09580915702E82369
:103970001CC0E82FF0E090915702EE0FFF1FE250BD
:10398000F14E222379F080916C03882359F08491C1
:10399000E82FE92BE093570280916B03882339F0DD
:1039A000E77703C0E491E095E923E093570281E0D3
:1039B00080936A0308956F70623051F028F4662393
:1039C00039F0613031F00895643011F0683011F44D
:1039D000FFCC6BCD08956F70623049F018F461111F
:1039E0000DC00BC0643049F0683041F406C022239A
:1039F00021F090916C03911101C022CD08951F9385
:103A0000CF93DF931F92CDB7DEB7182F862F807F1D
:103A100029F08093620181E080936A03113C09F4EC
:103A200088C0B8F5163BE0F4113B08F0ADC0133880
:103A300009F46DC050F4143008F4FBC0143708F4D6
:103A400053C0123809F45BC0F4C0143809F469C0DB
:103A500089E6810F893108F0ECC0812FA4DDEFC029
:103A6000183B09F4A8C050F4163B09F49EC0173B5C
:103A700009F0DFC08091670381509AC0193B09F4B7
:103A80009EC083E4810F833008F0D3C0812FBADD5C
:103A9000D6C01E3C09F46CC0B0F4193C09F45BC0FC
:103AA00048F4133C09F449C008F445C0183C09F433
:103AB00046C0BFC01C3C09F497C008F0A9C01A3C1E
:103AC00009F4BDC0B6C0183E38F4103E08F0AEC0D0
:103AD0001F3C09F086C050C080E1810F8A3008F099
:103AE000A8C0812F0BDEABC080916803882321F032
:103AF000812F6983D1DD6981812F5DDFA0C0809135
:103B0000580281FD9CC06091570289E307C08091F3
:103B1000580280FD94C06091570283E50E94E6122E
:103B20008EC08091580282FD8AC06091570287E45E
:103B3000F5CF3CD484C014D482C004D480C090910A
:103B40006F0381E0892780936F03811102C085E1B3
:103B50000BC085E154C090916B0381E0892780936D
:103B60006B03811103C085E037D369C085E047C08E
:103B700082E08093BE0163C08091870181115FC0A4
:103B800081E0809387015BC0EFE4E10FF0E0EE0F8E
:103B9000FF1FEC54FF4DE49180916603E82BE09306
:103BA000660381E080932C044AC0809167038F5F95
:103BB0008093670309C080917402815003C0809193
:103BC00074028F5F8093740290912D0480916C0336
:103BD000992321F090912B04981788F580932B045A
:103BE0002EC0812F75DD2BC09091680381E089275D
:103BF00080936803882329F01092730180E1CCD26E
:103C00001EC08091730181118093640180E1ACCF6B
:103C100080916803811113C060916401062E000C2D
:103C2000770B85E792E00E94331309C0812F26DECF
:103C300006C0612F70E040E084E40E94CD13109331
:103C400059020F90DF91CF911F9108951F93CF9349
:103C5000DF9300D01F92CDB7DEB7962F907F29F06B
:103C60001092620191E090936A03893B09F49DC030
:103C700008F040C0803BD0F4873908F085C0823816
:103C800009F45DC060F49CEF980F903708F0ACC069
:103C90000F900F900F90DF91CF911F919CCE8338A2
:103CA00009F455C0843809F461C09EC0863B09F40C
:103CB00072C0B0F4813B08F497C06FE4680FE62F40
:103CC000F0E0EE0FFF1FEC54FF4DE491E095809182
:103CD0006603E823E093660381E080932C0490C0A0
:103CE000873B09F45CC0883B09F07EC08091740278
:103CF0008F5F5EC08B3C70F4883C08F081C08D3BC8
:103D000008F472C0803CD0F19FE3980F933008F420
:103D100077C06AC0883E38F4803E08F04CC08C3CC6
:103D200008F06EC061C090E1980F9A3008F05CC056
:103D30000F900F900F90DF91CF911F911BCD80912D
:103D4000580281FF5DC06091570289E307C08091EE
:103D5000580280FF55C06091570283E50F900F9085
:103D60000F90DF91CF911F910C94E6128091580231
:103D700082FF46C06091570287E4F0CF10926E0335
:103D800081E0809363033CC00F900F900F90DF9110
:103D9000CF911F911FCC80916703815003C0809108
:103DA00067038F5F809367032BC0809174028150FB
:103DB0008093740225C0182F80916803882361F0D6
:103DC00080915902811308C080E02B834A83698364
:103DD00063DC69814A812B81812F0F900F900F90B6
:103DE000DF91CF911F917ACD682F70E040E085E49C
:103DF0000F900F900F90DF91CF911F910C94CD13E6
:103E00000F900F900F90DF91CF911F910895209107
:103E10005702227291E009F090E0209141042223A0
:103E200059F0992349F02091580220FF05C022EE55
:103E3000280F2A3008F4855C20913404222321F1D4
:103E4000833571F49091580281E08927809358025C
:103E500080FF03C080E0A0D11FC080E0BDD11CC0A6
:103E600027EA280F2B3080F420915802E82FF0E049
:103E7000EE0FFF1F20FF05C0992319F0E754F04E05
